:10F800000C94387C0C94557C0C94557C0C94557C51
:10F810000C94557C0C94557C0C94557C0C94557C24
:10F820000C94557C0C94557C0C94557C0C94557C14
:10F830000C94557C0C94557C0C94557C0C94557C04
:10F840000C94557C0C94557C0C94557C0C94557CF4
:10F850000C94557C0C94557C0C94557C0C94557CE4
:10F860000C94557C0C94557C0C94557C0C94557CD4
:10F8700011241FBECFEFD0E1DEBFCDBF11E0A0E06D
:10F88000B1E0ECE2FCEF02C005900D92A630B107AA
:10F89000D9F711E0A6E0B1E001C01D92AC30B1078C
:10F8A000E1F70E94727C0C94147E0C94007C982FDB
:10F8B0008091C00085FFFCCF9093C6000895809191
:10F8C000C00087FFFCCF8091C600089588B1807882
:10F8D00088B981E085BF15BEE0910601F09107016E
:10F8E000099508952F923F924F925F926F927F9267
:10F8F0008F929F92AF92BF92CF92DF92EF92FF9240
:10F900000F931F93CF93DF9304B603FE06C0E091DD
:10F910000601F0910701099508C088E10FB6F89437
:10F9200080936000109260000FBE1092C5008AE0C4
:10F930008093C40086E08093C20088E18093C10078
:10F9400082E60E94577C3F98479A379B05C081E624
:10F950000E94577C0E94667C80E70E94577C0E9430
:10F960005F7C863509F478C08735C8F48C3409F497
:10F970000BC18D3450F4823409F480C0853409F40D
:10F9800003C1813409F04EC128C0833509F45BC03E
:10F99000843509F44BC0803509F044C1F5C0853683
:10F9A00069F1863648F48136B1F0823609F45EC0DA
:10F9B000883509F037C157C0803709F452C0813704
:10F9C00020F4873609F02EC1E1C0833791F18437E6
:10F9D00009F028C136C089E5C0CF0E945F7C182F8E
:10F9E0000E945F7C912E882490E088299929909329
:10F9F000090180930801880F991F13C080E090E0EF
:10FA00000CC007B600FCFDCFF999FECF23E0FC0146
:10FA100020935700E89580509F4F48EF803094071F
:10FA200080F390930B0180930A01AEC00E945F7C2B
:10FA3000ABC089E00E94577C86E90E94577C8EE12A
:10FA40008CCF82E017C0C0E0D1E003C00E94577C99
:10FA5000219688818823D1F780E30E94577C82E336
:10FA60007CCF83E57ACF0E94667C8EC089E50E94B8
:10FA7000577C81E00E94577C80E06FCF0E945F7CC2
:10FA8000182F0E945F7C712E6624082F10E0062933
:10FA9000172981E00130180708F0C4C00E945F7C7C
:10FAA000863409F050C080910A0190910B01815079
:10FAB000984F18F080E00E94577CA0900A01B09007
:10FAC0000B0107B600FCFDCF6801D694C794750101
:10FAD000C0E0D0E016C00E945F7C082F0E945F7CCF
:10FAE000582E442410E00429152941E00801F701AB
:10FAF00040935700E895112482E090E0E80EF91E4B
:10FB00002196CC15DD0538F39601220F331F2A0DFF
:10FB10003B1D07B600FCFDCFF999FECF80910A018D
:10FB200090910B0145E0FC0140935700E89507B622
:10FB300000FCFDCF81E180935700E89530930B01E5
:10FB400020930A0121C0853409F06CC0C0E0D0E0E8
:10FB500018C00E945F7C2091080130910901F99939
:10FB6000FECF1FBA32BD21BD80BD0FB6F894FA9A00
:10FB7000F99A0FBE2F5F3F4F309309012093080180
:10FB80002196C017D10728F38DE0E7CE0E945F7C55
:10FB9000182F0E945F7C312E2224E82EFF24E228B9
:10FBA000F3280E945F7C8634E9F4C0E0D0E016C000
:10FBB000E0910A01F0910B0105911491802F0E94B0
:10FBC000577C812F0E94577C80910A0190910B01F4
:10FBD000029690930B0180930A012296CE15DF05C1
:10FBE00038F3BDCE8534F1F410E016C080910801E1
:10FBF00090910901F999FECF92BD81BDF89A80B527
:10FC00000E94577C80910801909109010196909380
:10FC10000901809308011F5F812F90E08E159F05D9
:0CFC200028F39DCE8FE399CEF894FFCF1F
:06FC2C0046444C20760066
:040000030000F80001
:00000001FF
